:100000000C9461000C9473000C9473000C947300B6
:100010000C9473000C9473000C9473000C94730094
:100020000C9473000C9473000C9473000C94730084
:100030000C9473000C9473000C9473000C94730074
:100040000C94A8000C9473000C9473000C9473002F
:100050000C9473000C9473000C9473000C94730054
:100060000C9473000C94730000000008000201005F
:100070000003040700000000000000000102040863
:100080001020408001020408102001020408102002
:10009000040404040404040402020202020203032E
:1000A00003030303000000002300260029000000D2
:1000B0000000250028002B0000000000240027007D
:1000C0002A0011241FBECFEFD8E0DEBFCDBF21E054
:1000D000A0E0B1E001C01D92A930B207E1F70E9493
:1000E0003A020C944A020C94000060E08BE00E94FB
:1000F000A10160E08DE00E94A10160E08CE00E941F
:10010000A10161E084E00C94A1018BE00E94100247
:10011000892BE9F48DE00E9410020197C1F48CE074
:100120000E941002892B21F460E084E00E94DA0131
:100130008CE00E941002019751F461E084E00E947B
:10014000DA0168EE73E080E090E00C941501089508
:100150001F920F920FB60F9211242F933F938F93FC
:100160009F93AF93BF938091010190910201A09161
:100170000301B09104013091000123E0230F2D37DA
:1001800020F40196A11DB11D05C026E8230F02969B
:10019000A11DB11D209300018093010190930201E4
:1001A000A0930301B0930401809105019091060191
:1001B000A0910701B09108010196A11DB11D809386
:1001C000050190930601A0930701B0930801BF9128
:1001D000AF919F918F913F912F910F900FBE0F90F4
:1001E0001F9018953FB7F8948091050190910601F2
:1001F000A0910701B091080126B5A89B05C02F3F2B
:1002000019F00196A11DB11D3FBF6627782F892FD8
:100210009A2F620F711D811D911D42E0660F771F9D
:10022000881F991F4A95D1F70895CF92DF92EF92D8
:10023000FF92CF93DF936B017C010E94F200EB01F0
:10024000C114D104E104F10489F00E9449020E9422
:10025000F2006C1B7D0B683E734090F381E0C81A7E
:10026000D108E108F108C851DC4FEACFDF91CF9106
:10027000FF90EF90DF90CF900895789484B58260DE
:1002800084BD84B5816084BD85B5826085BD85B53A
:10029000816085BDEEE6F0E0808181608083E1E8E9
:1002A000F0E0108280818260808380818160808321
:1002B000E0E8F0E0808181608083E1EBF0E0808124
:1002C00084608083E0EBF0E0808181608083EAE7F6
:1002D000F0E080818460808380818260808380817F
:1002E000816080838081806880831092C10008953E
:1002F000833081F028F4813099F08230A1F00895A4
:100300008730A9F08830B9F08430D1F48091800032
:100310008F7D03C0809180008F7780938000089547
:1003200084B58F7702C084B58F7D84BD0895809198
:10033000B0008F7703C08091B0008F7D8093B000B4
:100340000895CF93DF9390E0FC01E458FF4F249190
:10035000FC01E057FF4F8491882349F190E0880F1A
:10036000991FFC01E854FF4FA591B49182559F4F0E
:10037000FC01C591D4919FB7611108C0F8948C918C
:10038000209582238C93888182230AC0623051F4A5
:10039000F8948C91322F309583238C938881822B13
:1003A000888304C0F8948C91822B8C939FBFDF913B
:1003B000CF9108950F931F93CF93DF931F92CDB7E3
:1003C000DEB7282F30E0F901E859FF4F8491F90199
:1003D000E458FF4F1491F901E057FF4F04910023B7
:1003E000C9F0882321F069830E9478016981E02F98
:1003F000F0E0EE0FFF1FE255FF4FA591B4919FB7BC
:10040000F8948C91611103C01095812301C0812B58
:100410008C939FBF0F90DF91CF911F910F91089503
:10042000CF93DF93282F30E0F901E859FF4F8491F3
:10043000F901E458FF4FD491F901E057FF4FC491FF
:10044000CC2391F081110E947801EC2FF0E0EE0FA7
:10045000FF1FEC55FF4FA591B4912C912D2381E006
:1004600090E021F480E002C080E090E0DF91CF9145
:10047000089508950E943D010E9439020E9475006E
:10048000C0E0D0E00E9485002097E1F30E940000C8
:08049000F9CF0895F894FFCFA5
:00000001FF
